:020000040000FA
:06000000D43001303A2863
:08000800A000030EA100831209
:1000100005191028831601178312B23081002B288E
:1000200083160113831203140B190310A80DA90DD5
:10003000AA0DAB0DAC0DAC16FF302C02031D2B2806
:10004000FA302B02031D2B2831152A08AF0029088E
:10005000AE002808AD008B100B11210E8300A00EFE
:04006000200E090065
:0C007400203084008001840A80300402E7
:10008000031C3C281230B000C92183160C308505B2
:1000900087018312850187010730990000309A009B
:1000A000103083168E008312603083168F00831207
:1000B0000030831691009F008312C83083168100A0
:1000C000831231309000003083168C008312103080
:1000D0008B00AB2281018E018F010B118B100B1055
:1000E0008C018B17812031198420B30B7F280310DA
:1000F00085190314B90DF030390203192D210A2393
:10010000722864003210080031110130B7008B13DF
:100110002030370783169B001C141A088312A40092
:100120001030370783169B001C141A088312A30093
:10013000A6000230A6060030370783169B001C1469
:100140001A088312A200A7000130A7068B17321CE1
:10015000AF2822090339A200A309A409A50924088C
:100160002F02031D272923082E02031D27292208F9
:100170002D02031D272901303702031DC4283D1815
:10018000C4283D143E14E42102303702031DCD285B
:10019000BD18CD28BD143E14F02103303702031DD5
:1001A000D6283D19D6283D153E14FC2104303702CF
:1001B000031DDF28BD19DF28BD153E1408220530B8
:1001C0003702031DE8283D1AE8283D163E14142284
:1001D00006303702031DF128BD1AF128BD163E1462
:1001E000202207303702031DFA283D1BFA283D174D
:1001F0003E142C2208303702031D0329BD1B03299E
:10020000BD173E14372209303702031D0C295D1833
:100210000C295D143E1442220A303702031D1529B1
:10022000DD181529DD143E144D220B303702031D55
:100230001E295D191E295D153E1458220C30370207
:10024000031D2729DD192729DD153E146322B70A6E
:100250000D3037020318080087280130B600B300BC
:10026000B400B500B70085018701B1138120B30B3D
:100270007529031085190314B90DF03039020319DB
:100280009C29B40B75290130370203196F22023003
:10029000370203197422033037020319792204301C
:1002A000370203197E2205303702031983220630F4
:1002B0003702031988220730370203198D220830CC
:1002C00037020319922209303702031997220A30A4
:1002D000370203199C220B3037020319A1220C307C
:1002E00037020319A6229630B400311D3629311188
:1002F000321C7F292D090339AD00AE09AF092F1C2F
:1003000036298E018F010C1C36290C102E1E362921
:100310008B1320303707BB002F08BA00B4211030F0
:100320003707BB002E08BA00B42100303707BB00E6
:100330002D08BA00B4218B1785018701B70AB601D1
:100340000D303702031C3629AB2208003E1C080082
:100350003E101030BB003D08BA00B4213030BB0065
:100360005D08BA00B42108008B133A0883161C15E7
:100370009A0083123B0883169B0055309D00AA30DB
:100380009D009C1464009C18C2291C1183128B17B9
:100390000800831610309B001C141A088312BD003D
:1003A000831630309B001C141A088312DD00FF30C6
:1003B000C800CA15CB15CC15CD15CE15CF15D01547
:1003C000D115D215D3150800C130BD05FF30DD05AC
:1003D0005F140C30C405C0000030C2005E1008007D
:1003E000C230BD05FF30DD055F140330C405C00019
:1003F0000030C2005E100800C430BD05FF30DD05CE
:100400005F141330C405C0000030C2005E10080045
:10041000C830BD05FF30DD055F140930C405C000DC
:100420000030C2005E100800D030BD05FF30DD0591
:100430005F141930C405C0000030C200DE1008008F
:10044000E030BD05FF30DD055F140030C405C0009D
:100450000030C200DE1008007F30BD050030DD0531
:100460005F146030C505C1000030C3000800BF3014
:10047000BD050030DD055F141830C505C100003032
:10048000C30008003F30BD050130DD055F14983022
:10049000C505C1000030C30008003F30BD05023073
:1004A000DD055F144830C505C1000030C3000800F9
:1004B0003F30BD050430DD055F14C830C505C100FF
:1004C0000030C30008003F30BD050830DD055F1473
:1004D0000030C505C1000030C3000800080003302B
:1004E0008506003087060800303085060030870614
:1004F0000800303085060230870608001230850675
:100500000030870608001230850602308706080092
:10051000333085060230870608000030850630300B
:100520008706080000308506053087060800003081
:1005300085060D30870608000030850614308706D2
:100540000800003085061C3087060800003085064C
:100550003D30870608003D18E421BD18F0213D1903
:10056000FC21BD1908223D1A1422BD1A20223D1B70
:100570002C22BD1B37225D184222DD184D225D1949
:100580005822DD1963220800B601B301B4013C1CF6
:10059000CC2ABC01BC14CE2ABC013C143C08B600D9
:1005A0006400D22AD32AD42AD52AD62AFF30B41BF3
:1005B0008500B41F8501B30BD02AB40BD02A0310D9
:1005C000B60CB608031DD02A0030BB003C08BA00A8
:1005D000B421080005125C180516DC1C8512DC1815
:1005E00085165C1D05105C190514DC1D8510DC19D1
:1005F00085145C1E87105C1A8714DC1E0711DC1A38
:1006000007155C1F07105C1B0714DC1F8712DC1B1F
:10061000871608008F08031908008F0178308E00B4
:10062000C80F4E2DC80A4208C600C2014308C700C1
:10063000C301DE19422B441C422B461C332BCA1C1F
:10064000242BCA014A15502B4A1D292BCA01CA1551
:10065000502BCA1D2E2BCA014A16502B4A1E502B56
:10066000CA01CA14502B4A1D382BCA014A16502BF6
:10067000CA1D3D2BCA014A16502B4A1E502BCA01D7
:10068000CA14502BCA1C472BCA014A15502B4A1DAD
:100690004C2BCA01CA15502B4A1E502BCA014A15B1
:1006A000DE19792BC41C792BC61C6A2BCB1C5B2B47
:1006B000CB014B15872B4B1D602BCB01CB15872B0B
:1006C000CB1D652BCB014B16872B4B1E872BCB01EC
:1006D000CB14872B4B1D6F2BCB014B16872BCB1DC0
:1006E000742BCB014B16872B4B1E872BCB01CB14C6
:1006F000872BCB1C7E2BCB014B15872B4B1D832BC4
:10070000CB01CB15872B4B1E872BCB014B15DE194D
:10071000B02B441DB02B461DA12BCC1C922BCC0121
:100720004C15BE2B4C1D972BCC01CC15BE2BCC1DD4
:100730009C2BCC014C16BE2B4C1EBE2BCC01CC14DA
:10074000BE2B4C1DA62BCC014C16BE2BCC1DAB2BAF
:10075000CC014C16BE2B4C1EBE2BCC01CC14BE2B98
:10076000CC1CB52BCC014C15BE2B4C1DBA2BCC018F
:10077000CC15BE2B4C1EBE2BCC014C15DE19E82B24
:10078000C41DE82BC61DD92BCD1CCA2BCD014D1580
:100790005E13F62B4D1DCF2BCD01CD15F62BCD1DA8
:1007A000D42BCD014D16F62B4D1EF62BCD01CD14BD
:1007B000F62B4D1DDE2BCD014D16F62BCD1DE32B5B
:1007C000CD014D16F62B4D1EF62BCD01CD14F62B7B
:1007D000CD1CED2BCD014D15F62B4D1DF22BCD0172
:1007E000CD15F62B4D1EF62BCD014D15DE19212C06
:1007F0005E1B212C441E212C461E122CCE1C032CC9
:10080000CE014E152F2C4E1D082CCE01CE152F2CAF
:10081000CE1D0D2CCE014E162F2C4E1E2F2CCE0190
:10082000CE142F2C4E1D172CCE014E162F2CCE1D64
:100830001C2CCE014E162F2C4E1E2F2CCE01CE146A
:100840002F2CCE1C262CCE014E152F2C4E1D2B2CC2
:10085000CE01CE152F2C4E1E2F2CCE014E15DE199B
:10086000582CC51D582CC71D492CCF1C3A2CCF0124
:100870004F15662C4F1D3F2CCF01CF15662CCF1D79
:10088000442CCF014F16662C4F1E662CCF01CF147F
:10089000662C4F1D4E2CCF014F16662CCF1D532CAE
:1008A000CF014F16662C4F1E662CCF01CF14662C3D
:1008B000CF1C5D2CCF014F15662C4F1D622CCF0134
:1008C000CF15662C4F1E662CCF014F15DE198F2CCD
:1008D000451E8F2C471E802CD01C712CD00150152A
:1008E0009D2C501D762CD001D0159D2CD01D7B2C1D
:1008F000D00150169D2C501E9D2CD001D0149D2C43
:10090000501D852CD00150169D2CD01D8A2CD00155
:1009100050169D2C501E9D2CD001D0149D2CD01C07
:10092000942CD00150159D2C501D992CD001D01520
:100930009D2C501E9D2CD0015015DE19C62CC51EB5
:10094000C62CC71EB72CD11CA82CD1015115D42CF4
:10095000511DAD2CD101D115D42CD11DB22CD101FA
:100960005116D42C511ED42CD101D114D42C511D8C
:10097000BC2CD1015116D42CD11DC12CD101511642
:10098000D42C511ED42CD101D114D42CD11CCB2C5D
:10099000D1015115D42C511DD02CD101D115D42CFD
:1009A000511ED42CD1015115DE19FE2C451FFE2CF1
:1009B000471FEF2CD21CE02CD2015215DE130C2D58
:1009C000521DE52CD201D2150C2DD21DEA2CD201DC
:1009D00052160C2D521E0C2DD201D2140C2D521D6C
:1009E000F42CD20152160C2DD21DF92CD201521624
:1009F0000C2D521E0C2DD201D2140C2DD21C032D05
:100A0000D20152150C2D521D082DD201D2150C2DDC
:100A1000521E0C2DD2015215DE19372DDE1B372D3B
:100A2000C51F372DC71F282DD31C192DD3015315D2
:100A3000452D531D1E2DD301D315452DD31D232D1B
:100A4000D3015316452D531E452DD301D314452DE7
:100A5000531D2D2DD3015316452DD31D322DD301FA
:100A60005316452D531E452DD301D314452DD31CAC
:100A70003C2DD3015315452D531D412DD301D315C5
:100A8000452D531E452DD3015315A6214008C40002
:100A90004108C5005E18DE145E1CDE104808C9005F
:100AA0000C304A05031D05120C304B05031D851241
:100AB0000C304C05031D05100C304D05031D851031
:100AC0000C304E05031D87100C304F05031D071118
:100AD0000C305005031D07100C305105031D871203
:100AE0000C305205031D07120C305305031D8711EE
:100AF00049080E020318A82D12304A05031D0516D9
:100B000012304B05031D851612304C05031D0514CC
:100B100012304D05031D851412304E05031D871438
:100B200012304F05031D071512305005031D071421
:100B300012305105031D871612305205031D07168A
:100B400012305305031D8715FF30480203190800B2
:100B50008F08031D0800812049080E02031CA82DE0
:100B600018304A05031D051206304A05031D0516F7
:100B700018304B05031D851206304B05031D8516E5
:100B800018304C05031D051006304C05031D0514D7
:100B900018304D05031D851006304D05031D8514C5
:100BA00018304E05031D871006304E05031D8714AF
:100BB00018304F05031D071106304F05031D07159B
:100BC00018305005031D071006305005031D07148B
:100BD00018305105031D871206305105031D871675
:100BE00018305205031D071206305205031D071663
:100BF00018305305031D871106305305031D871553
:020C00000800EA
:084000000900030006000200A4
:02400E00CC33B1
:10420000010078007A007C007E007B0079007F004E
:104210007D007A0078007E007C007D007F007900C0
:104220000200F200F600FA00FE00F200F600FA00CA
:10423000FE00F200F600FA00FE00F200F600FA00BE
:10424000FF00050005000500050009000900090040
:1042500009000D000D000D000D00110011001100EE
:104260000100FF00FF00FF00FF00FF00FF00FF0054
:10427000FF00FF00FF00FF00FF00FF00FF00FF0046
:10428000FF007B00FF00FF00FF00FF00FF00FF00BA
:10429000FF00FF00FF00FF00FF00FF00FF00FF0026
:1042A000FF00FE00FF00FF00FF00FF00FF00FF0017
:1042B000FF00FF00FF00FF00FF00FF00FF00FF0006
:1042C000FF001100FF00FF00FF00FF00FF00FF00E4
:1042D000FF00FF00FF00FF00FF00FF00FF00FF00E6
:1042E000FF00FF00FF00FF00FF00FF00FF00FF00D6
:1042F000FF00FF00FF00FF00FF00FF00FF00DD00E8
:00000001FF
